:060000001BC049C07EC0D8
:10000600FCCFFBCFFACFF9CFF8CFF7CFF6CFF5CFAE
:10001600F4CFF3CFF2CFF1CFF0CFEFCFEECFEDCFDE
:100026000001020340004000000004006C012600AD
:100036000000F894EE27ECBBF1E0FBBFEBBFE5BF99
:10004600F8E1F1BDE1BD8DE0A2E0BB27ED938A9515
:10005600E9F780E094E0A0E6ED930197E9F7E0E3A5
:10006600F0E085919591009761F0A591B591059085
:100076001590BF01F00105900D920197E1F7FB0184
:10008600F0CFEFE5EDBFE4E0EEBFC0E6D1E09FC202
:1000960025D36F936FB76F937F938F939F936CB5B1
:1000A6007DB585B780FB4EF4609360017093610166
:1000B60065B76C7F626065BF11C060936201709323
:1000C60063018091600190916101681B790B6093D7
:1000D60064017093650165B7636065BF9F918F91F9
:1000E6007F916F916FBF6F9105B70170013011F469
:1000F600689401C0E89420F8F6D21895EFD26F9371
:100106006FB76F937F938F939F936CB57DB585B7CC
:1001160082FB4EF4609366017093670165B7637F57
:10012600686065BF11C06093680170936901809132
:10013600660190916701681B790B60936A01709361
:100146006B0165B76C6065BF9F918F917F916F91D1
:100156006FBF6F9105B70470043011F4689401C045
:10016600E89421F8C0D218956C9782E0A0E0B0E040
:10017600EAE2F0E0C6D3BBD2C6D271F420FE02C0DA
:1001860021FC01C007C0C5D2EC87FD87CAD2E8872B
:10019600F987F4CFCBD2F0CFAAD2CED2B4D259F4CB
:1001A60020FE02C021FC01C004C0B3D2EE87FF8747
:1001B600F7CFBCD2F3CF9BD2BFD2A5D259F420FE43
:1001C60002C021FC01C004C0A4D2E88BF98BF7CF92
:1001D600ADD2F3CF8CD2B0D296D259F420FE02C063
:1001E60021FC01C004C095D2EA8BFB8BF7CF9ED2CF
:1001F600F3CF7DD2A1D287D259F420FE02C021FCD2
:1002060001C004C086D2EC8BFD8BF7CF8FD2F3CF23
:100216006ED292D278D259F420FE02C021FC01C0DF
:1002260004C077D2EE8BFF8BF7CF80D2F3CF5FD2AD
:1002360083D269D259F420FE02C021FC01C004C059
:1002460068D2E88FF98FF7CF71D2F3CF50D274D23C
:100256005AD271F420FE02C021FC01C007C059D257
:10026600EA8FFB8F5ED2EA87FB87F4CF5FD2F0CFAF
:10027600E3E7E1BBE0E0E2BBAC85BD85EE85FF854B
:1002860060D2AC85BD85AE1BBF0BA0937001B09349
:100296007101EC85FD85AE85BF8556D25BD2EE85B4
:1002A600FF85A889B98950D25AD2E889F989AA89DD
:1002B600BB894AD259D2EA89FB89AC89BD8944D225
:1002C60058D2EC89FD89AE89BF893ED257D2EE89D4
:1002D600FF89A88DB98D38D256D2E88DF98DAA8DB1
:1002E600BB8D32D255D2A88DB98DEA8DFB8D29D220
:1002F600AA8DBB8DEA0FFB1F50D254D2A885B985B3
:1003060054D218F4E885F98501C04CD2EC83FD83FC
:1003160049D2A885B9854CD218F4E885F98501C07B
:1003260041D2EA83FB83AC81BD810BD2BED2EE8380
:10033600FF83AC81BD81EA0FFB1F3DD2AE81BF8139
:10034600EA81FB81FED13CD2F8943FD2A0E0B0E036
:10035600C1D2A2E0B0E03ED2BDD2A4E0B0E03FD22E
:10036600B9D2A6E0B0E040D2B5D2A8E0B0E041D222
:10037600B1D2AAE0B0E042D2ADD2ACE0B0E043D216
:10038600A9D2AEE0B0E044D2A5D2A0E1B0E045D219
:10039600A1D248D2A2E1B0E09DD2A4E1B0E047D21A
:1003A60099D2E8EEF3E0FA93EA9373D2E3E3E1BB82
:1003B60078946C960895219781E0A0E0B0E0EEE293
:1003C600F0E09FD22FD238D2F0D108F051C0E1E050
:1003D60038D220F4FFD13CD2E8D108F003C03DD298
:1003E600E1E048D2F7D149D218F4F9D148D208F061
:1003F60003C033D2E2E03ED2F2D13FD218F4F4D1B8
:100406003ED208F003C029D2E3E034D2EDD135D292
:1004160018F4EFD134D208F003C01FD2E4E02AD298
:10042600E8D12BD218F4EAD12AD208F003C015D2AB
:10043600E5E020D2E3D121D218F4E5D120D208F0AC
:1004460003C00BD2E6E016D2DED117D218F4E0D103
:1004560016D208F003C001D2E7E00CD2D9D10DD2F2
:1004660018F4DBD10CD208F003C0F7D1E8E002D2D1
:10047600DED1E2D19DD108F050C0E2E0E2D118F41D
:10048600A9D1FDD108F003C0E8D1E9E0F3D1A2D1AA
:10049600F4D118F4A4D1F3D108F003C0DED1EAE018
:1004A600E9D19DD1EAD118F49FD1E9D108F003C072
:1004B600D4D1EBE0DFD198D1E0D118F49AD1DFD1D5
:1004C60008F003C0CAD1ECE0D5D193D1D6D118F447
:1004D60095D1D5D108F003C0C0D1EDE0CBD18ED1F6
:1004E600CCD118F490D1CBD108F003C0B6D1EEE050
:1004F600C1D189D1C2D118F48BD1C1D108F003C0C2
:10050600ACD1EFE0B7D184D1B8D118F486D1B7D148
:1005160008F003C0A2D1E0E1ADD1E881E03021F4DA
:10052600B0D1E0E8E2BB51C0ACD1E0E0E2BBE09183
:100536006D01ABD141F4E0916E01A7D121F4E091B8
:100546006F01A3D109F041C0E0916C01E13011F4D3
:10055600C09A3BC0E23011F4C19A37C0E33011F4BF
:10056600C29A33C0E43011F4C39A2FC0E53011F4B7
:10057600C49A2BC0E63011F4C59A27C0E73011F4AF
:10058600A89A23C0E83011F4A99A1FC0E93011F4E3
:10059600AA9A1BC0EA3011F4AB9A17C0EB3011F4DB
:1005A600AC9A13C0EC3011F4AD9A0FC0ED3011F4D3
:1005B600909A0BC0EE3011F4919A07C0EF3011F407
:1005C600949A03C0E03109F4959A2196089500E0C3
:1005D600E0E0E8BBEFE3E7BBE0E0E5BBEFE3E4BB6D
:1005E600E0ECE2BBE3E3E1BBE0E0E3BFE2BFEFBD8B
:1005F600E2E0EEBDE0E0EDBDECBDE7BDE6BDEBBD86
:10060600EABDE9BDE8BDE2BDE5BDE4BDE3BDEBB7CE
:10061600E06CEBBFEFE0E5BFE0ECEABFE0E0E9BF8E
:10062600E0E8E8B9E0E0E0BFA0E0B0E043D1E09365
:100636007001F0937101A2E0B0E03CD18BD0A4E050
:10064600B0E038D18CD0A6E0B0E034D18DD0A8E0AF
:10065600B0E030D18ED0AAE0B0E02CD18FD0ACE0A3
:10066600B0E028D190D0AEE0B0E024D191D0A0E1A6
:10067600B0E020D192D0A2E1B0E01CD19CD0A4E1A0
:10068600B0E018D19DD07894E0B3E0780E2F00301A
:1006960009F46ADDE3EBE1BBE0ECE2BB20FE02C05D
:1006A60021FC01C019C0E89420F821F8D1D0AB385C
:1006B600E2E0BE0778F0CCD0A43CE9E0BE0750F4F7
:1006C600BBD0AB38E2E0BE0728F0B6D0A43CE9E0E8
:1006D600BE0708F001C06FDEE1CFFFCFEA93EFB7A8
:1006E6000A9300E008950991EFBFE9910895E3E7C1
:1006F600E1BBE0E0E2BBE8EEF3E0FA93EA93C9D0AF
:10070600E3E3E1BB0895A881B981A034E0E0BE0728
:100716000895E89420F821F8E0916401F0916501CC
:100726000895E0916A01F0916B010895E0B3E074D9
:10073600F0E0E883F9830895E0E4F0E0E883F983E4
:100746000895EA1BFB0B0895AE0FBF1FFD01F6953A
:10075600E7950895E0937201F09373010895E0938D
:100766007401F09375010895E0937601F093770193
:100776000895E0937801F09379010895E0937A0162
:10078600F0937B010895E0937C01F0937D01089539
:10079600E0937E01F0937F010895E0938001F0934A
:1007A60081010895EA85FB850895AE17BF07089570
:1007B600EA17FB070895E0938201F09383010895F9
:1007C600E0938401F09385010895E0917001F09122
:1007D60071010895E0917201F09173010895E0911D
:1007E6007401F09175010895E0917601F091770119
:1007F6000895E0917801F09179010895E0917A01E8
:10080600F0917B010895E0917C01F0917D010895BE
:10081600E0917E01F0917F010895E0918001F091D1
:1008260081010895E0918201F09183010895E0919C
:100836008401F09185010895A0916A01B0916B0140
:100846000895E883C2DFA0916401B0916501B0CF3D
:10085600A0916401B09165010895E0916E01E09365
:100866006F01E0916D01E0936E01E0916C01E09300
:100876006D010895E0936C010895EADF99CFE8DFF2
:1008860094CFE0E0E8BBE5BB0895A0916C01EA17C0
:100896000895E991F991309639F080ED97E0019746
:1008A600F1F7A8953197C9F70895F695E795F69566
:1008B600E7950895119602D0FE2F1197E199FECF84
:1008C600FF93FFB7F894AEBBBFBBE09AEDB3FFBF93
:1008D600FF91089507D01196EF93EF2F03D0EF9174
:1008E60011970895E199FECF9FB7F894AEBBBFBBB1
:1008F600E09A8DB3E81719F0EDBBE29AE19A9FBF33
:100906000895AC0FBD1F05900D928A95E1F70895E5
:00000001FF
